:020000040000FA
:100000005DEF17F0120012000EEF00F01200010079
:10001000182F0000600000009E000000DACFE4FF0F
:10002000E2CFDAFFE9CFE4FFEACFE4FFF6CFE4FF67
:10003000F7CFE4FFF5CFE4FFF3CFE4FFF4CFE4FF25
:10004000FACFE4FF00EE18F0140EE80403E3EECF5D
:10005000E4FFFBD700EE00F0180EE80403E3EECF58
:10006000E4FFFBD7E6529EAA3BD0D3EC16F0010189
:10007000616FABA406D0AB9EAB8E616B642B000EA0
:100080006523ABA206D0AB98AB88616B642B000EE6
:1000900065230D0E615D17E0400E96AF02D0D8903B
:1000A00003D0955D000E96590EE2BD0E9525E96EC2
:1000B000000E9621EA6E61C1EFFF952B000E96238C
:1000C000626B636B0CD0BD0E9525E96E000E962118
:1000D000EA6EEF6A010E626F636B956B966B9E9A88
:1000E0009EA432D0BECF6CF1BFCF6DF101016E6B1B
:1000F0006F6B6C0EE96E010EEA6E7051EE5C715121
:10010000EE587251EE587351EE5806E2FF0E6C270E
:100110006D23000E6E236F23700EE96E010EEA6EE2
:10012000EE506C5D6C6FEE506D596D6FEE506E5908
:100130006E6FEE506F596F6FBECF70F1BFCF71F120
:10014000726B736B94859E94E55200EE17F0180E57
:10015000E80403E3E5CFEDFFFBD700EE2BF0140E30
:10016000E80403E3E5CFEDFFFBD7E5CFFAFFE5CFEA
:10017000F4FFE5CFF3FFE5CFF5FFE5CFF7FFE5CFE0
:10018000F6FFE5CFEAFFE5CFE9FFE5CFDAFF1100A3
:10019000D9CFE6FFE1CFD9FFFB0EDBCF1DF0FC0E80
:1001A000DBCF1EF0FD0EDBCF1FF0FE0EDBCF20F00D
:1001B0002034000E201809E6D880000E1D54000ED1
:1001C0001E54000E1F54000E20540CE2D950FB0F99
:1001D000E96EFF0EDA20EA6EEE06000EEE5AEE5AD7
:1001E000EE5ADAD7E552E7CFD9FF1200700ED36E80
:1001F000330EE66EE66A7C0EE66E3EEC16F0E552D5
:10020000E552E5521200D9CFE6FFE1CFD9FF020E49
:10021000E126DE6ADD6AFD0EDBCFE9FFFE0EDBCFF5
:10022000EAFFEF5016E0FD0EDBCFE9FFFE0EDBCF5D
:10023000EAFFEF50E66EE66A1FD8E552E552DF2A84
:10024000010E01E3DB2AFD0EDB2AFE0E01E3DB2AB1
:10025000E2D7DECF00F0DDCF01F000C0F3FF01C038
:10026000F4FF020EE15C03E200D0E16AE552E16EC8
:10027000E552E7CFD9FF1200D9CFE6FFE1CFD9FF92
:10028000ACA2FED7FD0EDBCFE6FF0EEC17F0E55279
:10029000E552E7CFD9FF12000D0EE66EE66AECDFFD
:1002A000E552E5520A0EE66EE66AE6DFE552E552F1
:1002B0001200D9CFE6FFE1CFD9FF0A0EE1260101F6
:1002C000AC0E446F000E456FFC0EDBCF00F0010E4C
:1002D000E76E0018E8AE02D0003403D0E750D880B3
:1002E000005401E2DBD0FC0EDB5028E1FD0EDBCF39
:1002F00000F0FE0EDBCF01F0060E00C0DBFF070EA4
:1003000001C0DBFF080EDB6A090EDB6A44C1E6FFB1
:1003100045C1E6FFD950060FE96EDACFEAFFEECF0E
:10032000E6FFEECFE6FFEECFE6FFEFCFE6FF18ECFD
:1003300014F0006E060EE15E005010D044C1E6FFDE
:1003400045C1E6FFFD0EDBCFE6FFFE0EDBCFE6FF8D
:100350007EEC13F0E552E552E552E552010194AD11
:1003600084D0AC0EE66E000EE66E8BEC15F0E55216
:10037000E552020EF3CFDBFF030EF4CFDBFFDE6AA4
:10038000DD6ADECF00F0DDCF01F0020EDBCF02F040
:10039000030EDBCF03F00250005C035001582EE245
:1003A000020EDBCF02F0030EDBCF03F0DE50025C67
:1003B000E96EDD500358EA6EE906000EEA5AAC0E0B
:1003C000E926000EEA22EF50E66EFC0EDB50040F29
:1003D000006E016A00BE0168DE50005CE96EDD500F
:1003E0000158EA6EAC0EE926000EEA22E552E7500B
:1003F000EF6EDF2A010E01E3DB2AC3D7DE6ADD6A76
:10040000DECF00F0DDCF01F0FC0EDB50050F046EF7
:10041000056A04BE0568020EDB50045C026E030E22
:10042000DB500558036E0250005C035001581DE27A
:10043000010194A90BD0DECFE9FFDDCFEAFFAC0EBE
:10044000E926000EEA22300EEF6E0AD0DECFE9FF79
:10045000DDCFEAFFAC0EE926000EEA22200EEF6E99
:10046000DF2A010E01E3DB2ACBD7FC0EDB50050FA0
:10047000E96EEA6AE9BEEA68AC0EE926000EEA22F5
:10048000EF6A44C1E6FF45C1E6FFBDDEE552E55235
:10049000020EF3CFDBFF030EF4CFDBFF0A0EE15CAD
:1004A00002E2E16AE552E16EE552E7CFD9FF1200C0
:1004B000D9CFE6FFE1CFD9FF0E0EE126F90EDBCF53
:1004C000DEFFDBCFDDFFF80EDBCF02F0000EE76EC4
:1004D0000218E8AE02D0023403D0E750D8800254AC
:1004E00002E3070E12D0F80EDBCF03F0160EE76E14
:1004F0000318E8AE02D0033403D0E750D880035489
:1005000002E2170E02D0F80EDB28006E016A00BE70
:100510000168080E00C0DBFF090E01C0DBFF020E00
:10052000DB6A030EDB6AFB0EDBCF00F0FC0EDBCFD9
:1005300001F0FD0EDBCF02F0FE0EDBCF03F0226AEE
:10054000236A246A256A00C01DF001C01EF002C0A3
:100550001FF003C020F06DEC12F0010A33E1F90E38
:10056000DBCFE9FFDB2AFA0EDBCFEAFF01E3DB2A70
:100570002D0EEF6EFB0EDBCF00F0FC0EDBCF01F09B
:10058000FD0EDBCF02F0FE0EDBCF03F0226A236A02
:10059000800E246EBF0E256E00C01DF001C01EF03F
:1005A00002C01FF003C020F091EC11F0FB0E1DC043
:1005B000DBFFFC0E1EC0DBFFFD0E1FC0DBFFFE0ECF
:1005C00020C0DBFFFB0EDBCF00F0FC0EDBCF01F029
:1005D000FD0EDBCF02F0FE0EDBCF03F0226A236AB2
:1005E000246A256A00C01DF001C01EF002C01FF081
:1005F00003C020F064EC12F0010A4AE1FB0EDBCFED
:1006000000F0FC0EDBCF01F0FD0EDBCF02F0FE0EA2
:10061000DBCF03F0226A236A800E246E3F0E256E24
:1006200000C01DF001C01EF002C01FF003C020F08A
:100630006DEC12F0010A2CE1006A016A200E026ED4
:10064000410E036ED950FB0FE96EFF0EDA20EA6E01
:10065000EECF1DF0EECF1EF0EECF1FF0EFCF20F06B
:1006600000C022F001C023F002C024F003C025F036
:1006700091EC11F020C0EDFF1FC0EDFF1EC0EDFF9B
:100680001DC0EFFF020EDB06030E01E2DB06B6D74C
:10069000FB0EDBCF00F0FC0EDBCF01F0FD0EDBCF5D
:1006A00002F0FE0EDBCF03F0226A236A200E246ED6
:1006B000410E256E00C01DF001C01EF002C01FF0EB
:1006C00003C020F06DEC12F0010A2EE0FB0EDBCF30
:1006D00000F0FC0EDBCF01F0FD0EDBCF02F0FE0ED2
:1006E000DBCF03F0226A236A200E246E410E256EB2
:1006F00000C01DF001C01EF002C01FF003C020F0BA
:100700003EEC11F0FB0E1DC0DBFFFC0E1EC0DBFF3C
:10071000FD0E1FC0DBFFFE0E20C0DBFF020EDB2A3A
:10072000030E01E3DB2AB4D7020EDBCF00F0030E89
:10073000DBCF01F0D950080FE96EDACFEAFF0050A5
:10074000EE260150ED22010EF36E040EF3CFDBFF17
:10075000050EDB6A040EDBCF1EF0050EDBCF1FF0AB
:1007600079EC10F00A0E1DC0DBFF0B0E1EC0DBFF84
:100770000C0E1FC0DBFF0D0E20C0DBFF040EDBCF15
:1007800000F0050EDBCF01F0080EDBCF02F0090E02
:10079000DBCF03F001500318E8AE02D0033404D0DD
:1007A0000250005C035001582EE20A0EDBCF00F02D
:1007B0000B0EDBCF01F00C0EDBCF02F00D0EDBCF0A
:1007C00003F0226A236A200E246E410E256E00C0BB
:1007D0001DF001C01EF002C01FF003C020F03EEC6F
:1007E00011F00A0E1DC0DBFF0B0E1EC0DBFF0C0E4E
:1007F0001FC0DBFF0D0E20C0DBFF040EDB2A050E41
:1008000001E3DB2ABBD70A0EDBCF04F00B0EDBCFF4
:1008100005F00C0EDBCF06F00D0EDBCF07F0226AE1
:10082000236A246A400E256E04C01DF005C01EF028
:1008300006C01FF007C020F03EEC11F01DC000F014
:100840001EC001F01FC002F020C003F0D950FB0F02
:10085000E96EFF0EDA20EA6EEECF1DF0EECF1EF04D
:10086000EECF1FF0EFCF20F000C022F001C023F048
:1008700002C024F003C025F0A8EC10F020C0EDFF6A
:100880001FC0EDFF1EC0EDFF1DC0EFFFFB0EDBCF55
:1008900000F0FC0EDBCF01F0FD0EDBCF02F0FE0E10
:1008A000DBCF03F0226A236A200E246E410E256EF0
:1008B00000C01DF001C01EF002C01FF003C020F0F8
:1008C0006DEC12F0010A13E0FB0EDB6AFC0EDB6A32
:1008D000800EF36EFD0EF3CFDBFF3F0EF36EFE0EC8
:1008E000F3CFDBFF020EDB2A030E01E3DB2A020E4D
:1008F000DBCF00F0030EDBCF01F00001800E01140E
:100900005FE0F90EDBCFE9FFDB2AFA0EDBCFEAFF6F
:1009100001E3DB2A300EEF6EF90EDBCFE9FFDB2AB5
:10092000FA0EDBCFEAFF01E3DB2A2E0EEF6E080E94
:10093000DBCF00F0090EDBCF01F0800E011414E0D4
:10094000020EDBCF02F0030EDBCF03F0080EDB500C
:10095000025C006E090EDB500358016E020E00C0EF
:10096000DBFF030E01C0DBFF040EDB68050EDB6856
:10097000040EDBCF00F0050EDBCF01F0020EDBCF63
:1009800002F0030EDBCF03F003500118E8AE02D0F3
:10099000013404D00050025C0150035811E2F90EFA
:1009A000DBCFE9FFDB2AFA0EDBCFEAFF01E3DB2A2C
:1009B000300EEF6E040EDB06050E01E2DB06D8D723
:1009C000040EDB6A050EDB6A040EDBCF00F0050EB9
:1009D000DBCF01F0080EDBCF02F0090EDBCF03F016
:1009E00001500318E8AE02D0033404D00250005C7A
:1009F0000350015801E3ACD0FB0EDBCF1DF0FC0E21
:100A0000DBCF1EF0FD0EDBCF1FF0FE0EDBCF20F0A4
:100A1000FEEC11F0060E1EC0DBFF070E1FC0DBFF51
:100A2000300EE76E060EDBCF00F0070EDBCF01F0D5
:100A3000E7500026000E0122F90EDBCFE9FFDB2A8A
:100A4000FA0EDBCFEAFF01E3DB2A00C0EFFF040E62
:100A5000DBCF00F0050EDBCF01F0020EDB500018FB
:100A600003E1030EDB5001180BE1F90EDBCFE9FFC8
:100A7000DB2AFA0EDBCFEAFF01E3DB2A2E0EEF6E54
:100A8000060EDBCF1EF0070EDBCF1FF079EC10F067
:100A90000A0E1DC0DBFF0B0E1EC0DBFF0C0E1FC0BD
:100AA000DBFF0D0E20C0DBFF1DC000F01EC001F0FB
:100AB0001FC002F020C003F0D950FB0FE96EFF0EFB
:100AC000DA20EA6EEECF1DF0EECF1EF0EECF1FF073
:100AD000EFCF20F000C022F001C023F002C024F0CC
:100AE00003C025F0A7EC10F020C0EDFF1FC0EDFF04
:100AF0001EC0EDFF1DC0EFFF006A016A200E026EEE
:100B0000410E036ED950FB0FE96EFF0EDA20EA6E3C
:100B1000EECF1DF0EECF1EF0EECF1FF0EFCF20F0A6
:100B200000C022F001C023F002C024F003C025F071
:100B300091EC11F020C0EDFF1FC0EDFF1EC0EDFFD6
:100B40001DC0EFFF040EDB2A050E01E3DB2A3CD7B4
:100B5000F90EDBCFE9FFFA0EDBCFEAFFEF6ADECF5B
:100B600000F0DDCF01F000C0F3FF01C0F4FF0E0E76
:100B7000E15C03E200D0E16AE552E16EE552E7CFC5
:100B8000D9FF1200D9CFE6FFE1CFD9FF060EE1264B
:100B90000101949DFB0EDBCF1DF0FC0EDBCF1EF0A0
:100BA000FD0EDBCF1FF0FE0EDBCF20F02DEC12F0A0
:100BB0001CC0DEFF1DC0DEFF1EC0DEFF1FC0DDFF4C
:100BC000DD52DD52FB0EDBCF04F0FC0EDBCF05F077
:100BD000FD0EDBCF06F0FE0EDBCF07F0F90EDBCF0C
:100BE0001EF0FA0EDBCF1FF079EC10F01DC008F0FC
:100BF0001EC009F01FC00AF020C00BF008C022F090
:100C000009C023F00AC024F00BC025F004C01DF079
:100C100005C01EF006C01FF007C020F091EC11F0D7
:100C20001DC000F01EC001F01FC002F020C003F084
:100C3000F90EDBCF14F0FA0EDBCF15F0166A176A47
:100C400015AE02D01668176814C01CF015C01DF050
:100C500016C01EF017C01FF0DFCF21F0010EDBCF52
:100C600022F0020EDBCF23F0030EDBCF24F077EC73
:100C700016F018C010F019C011F01AC012F01BC005
:100C800013F010C01CF011C01DF012C01EF013C0F4
:100C90001FF08EEC10F01DC00CF01EC00DF01FC038
:100CA0000EF020C00FF00CC022F00DC023F00EC0DB
:100CB00024F00FC025F000C01DF001C01EF002C0DE
:100CC0001FF003C020F0A7EC10F0FEEC11F0040EB2
:100CD0001EC0DBFF050E1FC0DBFF6C0EE66E000EB4
:100CE000E66ED9CFE9FFDACFEAFFEECFE6FFEECF2F
:100CF000E6FFEECFE6FFEFCFE6FF18EC14F0006E54
:100D0000060EE15E00506C0EE66E000EE66E03EC21
:100D100001F0E552E552F3CF5BF1F4CF5CF12E0E1A
:100D2000E66EE66A3CEC01F0E552E552F80EDBCFE8
:100D3000E6FFE66A040EDBCFE6FF050EDBCFE6FF3B
:100D400059EC01F0E552E552E552E552060EE15C40
:100D500002E2E16AE552E16EE552E7CFD9FF120007
:100D6000D9CFE6FFE1CFD9FFE652800EDF6EDF502C
:100D7000000817E2FE0EDB50DF1408E0310EE66ECD
:100D8000E66A3CEC01F0E552E55207D0300EE66E23
:100D9000E66A3CEC01F0E552E552DF407F0BDF6E86
:100DA000E6D7E552E552E7CFD9FF1200D9CFE6FFEB
:100DB000E1CFD9FF020EE126FE0EDB50F00BE83842
:100DC0000F0B300FDF6EDF50390803E2070EDF2410
:100DD000DF6EFE0EDB500F0B300FE76E010EE7CF1C
:100DE000DBFFDB5039080AE2070E006E010EDBCF95
:100DF000E7FF0050E726010EE7CFDBFFDFCFE6FF7E
:100E0000E66A3CEC01F0E552E552010EDBCFE6FF6D
:100E1000E66A3CEC01F0E552E552680EE66EE66AE1
:100E20003CEC01F0E552E552020EE15C02E2E16ABF
:100E3000E552E16EE552E7CFD9FF1200D9CFE6FFC8
:100E4000E1CFD9FF020EE126DE6ADD6ADECF00F0D7
:100E5000DDCF01F0FE0EDB50000101AE02D0D890D4
:100E600003D0005C000E01580CE2200EE66EE66A2C
:100E70003CEC01F0E552E552DF2A010E01E3DB2AEA
:100E8000E5D7020EE15C02E2E16AE552E16EE5526D
:100E9000E7CFD9FF1200D9CFE6FFE1CFD9FFFE0E91
:100EA000DB50A96EA69EA69CA680F40EE66E010EEF
:100EB000E66EE66AE66AC8EC00F0E552E552E552F5
:100EC000E552A85000D0E552E7CFD9FF1200D9CFA4
:100ED000E6FFE1CFD9FFFE0EDB50A96EFD0EDB5021
:100EE000A86EA69EA684550EA76EAA0EA76EA68211
:100EF000A1A8FED7A198A694E552E7CFD9FF12008A
:100F0000D9CFE6FFE1CFD9FFFB0EDBCFE9FFFC0E27
:100F1000DBCFEAFFEF501AE0FB0EDBCFE9FFDB2A65
:100F2000FC0EDBCFEAFF01E3DB2AEF50E66EFD0E9D
:100F3000DBCF00F0DB2AFE0EDBCF01F001E3DB2A82
:100F40000050E66EC4DFE552E552DED7E552E7CF4A
:100F5000D9FF1200D9CFE6FFE1CFD9FF020EE1267B
:100F6000FD0EDBCFE6FF97DFE552DE6EDD6AD9CFFF
:100F7000E9FFDACFEAFFEE50ED1001E121D0DFCF3B
:100F8000E6FFE66A3CEC01F0E552E552FD0EDB2A95
:100F9000FE0E01E3DB2AFD0EDBCF00F0FE0EDBCF01
:100FA00001F0013404E20050FF08000E015401E298
:100FB00007D0D9CFE9FFDACFEAFFEE50ED10D0E14C
:100FC000980EE66E3A0EE66EE66AE66AC8EC00F047
:100FD000E552E552E552E552020EE15C02E2E16AB9
:100FE000E552E16EE552E7CFD9FF12000F01396BF0
:100FF0008168936893809382939493869388938A6D
:10100000938C938EC26A070EC16E926E896A3A6B98
:101010008268860E946E94909482948494969498A8
:10102000949A949C948E12009484BD96BD84BD8243
:10103000BD909D84D08EF29E1200CD9ACD98CD9613
:10104000CD94CD82CD90D08E000EE66EE66AF2ECA5
:1010500016F0E552E5529E909F809D901200700E12
:10106000D36E9B6A9B9CC2DF89980101466BAC0ED4
:10107000446F000E456F646B656B626B636B666BF0
:10108000676B0001BD6BF6EC00F00101949F9EAA16
:1010900005D0D3EC16F00101566FF9D7AB889D8AC5
:1010A0009F8AD08EF28CF28E200EE66E4E0EE66E89
:1010B000E66AE66AC8EC00F0E552E552E552E55210
:1010C00089880C0EE66EE66A3CEC01F0E552E552CA
:1010D000900EE66ED00EE66E030EE66EE66AC8EC83
:1010E00000F0E552E552E552E55201014B6B4C6BC5
:1010F000006B016B4CEC01F001016C0E026F000EF5
:10110000036F02C1E6FF03C1E6FF03EC01F0E55205
:10111000E552F3CF5BF1F4CF5CF14CEC01F001014F
:101120006C0E026F000E036F62C000F063C001F02E
:10113000026A00C0E6FF01C0E6FF02C0E6FF02C18E
:10114000E6FF03C1E6FF72EC15F0036E050EE15EEB
:10115000035002C1E6FF03C1E6FF03EC01F0E552D4
:10116000E552F3CF5BF1F4CF5CF1E80EE66E030ECF
:10117000E66EE66AE66AC8EC00F0E552E552E55232
:10118000E552000EE66EE66AE5DEE552E552200E17
:10119000E66EE66ADFDEE552E552600EE66EE66A6E
:1011A000D9DEE552E552A00EE66EE66AD3DEE552E0
:1011B000E552C00EE66EE66ACDDEE552E5524CEC35
:1011C00001F0100EE66E270EE66EE66AE66AC8ECDF
:1011D00000F0E552E552E552E55268C000F069C002
:1011E00001F0026A00C0E6FF01C0E6FF02C0E6FFB0
:1011F00002C1E6FF03C1E6FF72EC15F0036E050EB7
:10120000E15E035002C1E6FF03C1E6FF03EC01F01B
:10121000E552E552F3CF5BF1F4CF5CF14CEC01F019
:101220006AC000F06BC001F0026A00C0E6FF01C0B6
:10123000E6FF02C0E6FF02C1E6FF03C1E6FF72EC73
:1012400015F0036E050EE15E035002C1E6FF03C117
:10125000E6FF03EC01F0E552E552F3CF5BF1F4CF8A
:101260005CF14CEC01F001019495E7DEDDDE01015B
:10127000686B696B786979697A697B69746B756B7E
:10128000766B776B6C0E026F000E036F6C6B6D6B81
:101290006E6B6F6B6C0E026F000E036F9E90F28C84
:1012A000F28ECD80010E621901E1635116E1CD90FD
:1012B000BD0EE66E000EE66E03EC01F0E552E5525F
:1012C000F3CF5BF1F4CF5CF10101626B636B000162
:1012D000BD6B0101666B676BCD809E90949594A564
:1012E000FED76C0EE96E010EEA6E7C51EE247C6F27
:1012F0007D51EE207D6F7E51EE207E6F7F51EE207E
:101300007F6F68C100F069C101F0640E236E246A2A
:1013100000C01EF001C01FF025EC17F01AC000F04D
:101320001BC001F00050011001E0CAD07CC11CF0CC
:101330007DC11DF07EC11EF07FC11FF08CEC10F04E
:101340001DC000F01EC001F01FC002F020C003F05D
:10135000226A236AC80E246E420E256E00C01DF05C
:1013600001C01EF002C01FF003C020F03EEC11F0DF
:101370001DC084F11EC085F11FC086F120C087F119
:10138000C00E006EE10E016EE40E026E4B0E036E97
:1013900084C122F085C123F086C124F087C125F0E5
:1013A00000C01DF001C01EF002C01FF003C020F0FD
:1013B0003EEC11F01DC088F11EC089F11FC08AF1FA
:1013C00020C08BF1006A240E016E740E026E4B0E6B
:1013D000036E84C122F085C123F086C124F087C149
:1013E00025F000C01DF001C01EF002C01FF003C0B8
:1013F00020F03EEC11F01DC08CF11EC08DF11FC01D
:101400008EF120C08FF1010EE66E240EE66E010E05
:10141000E66E88C1E6FF89C1E6FF8AC1E6FF8BC19F
:10142000E6FF58EC02F0026E070EE15E0250F3CFC9
:1014300000F0F4CF01F000C0E6FF01C0E6FF010EAE
:10144000E66E040EE66E010EE66E8CC1E6FF8DC1FF
:10145000E6FF8EC1E6FF8FC1E6FF58EC02F0056E95
:10146000070EE15E0550F3CF03F0F4CF04F003C0A4
:10147000E6FF04C0E6FFF20E066E2E0E076E086A47
:1014800006C0E6FF07C0E6FF08C0E6FFFE0EE66EF8
:10149000E66824EC15F0096E090EE15E0950F3CF01
:1014A0005BF1F4CF5CF10101786979697A697B6954
:1014B000746B756B766B776B7C6B7D6B7E6B7F6B08
:1014C0000101682B000E6923EDD61200A2EC0FF08B
:1014D000FB0EDBCFF3FFDB06F35000090AE0F0EC74
:1014E0000FF0FA0E5BEC10F0F3E1011CF1E1010EDC
:1014F00001D0000ED1EF0FF0A2EC0FF03B0EE12473
:1015000002E3E168E652E16E010EDB6A020EDB6A7D
:10151000F90EDBCFF6FFFA0EDBCFF7FFFB0EDBCFCA
:10152000F8FF0800F550DF6EDF5002E1F5EF0EF036
:10153000250EDF5C02E0E8EF0EF0030EDB6A040E1E
:10154000DB6A050EDB6A060EDB6A070EDB6A0AEC55
:101550000FF02D0EDF5C0CE02B0EDF5C09E0200E9F
:10156000DF5C06E0230EDF5C03E0300EDF5C1AE197
:10157000DF50300A14E0130A0FE0030A0AE00B0AF6
:1015800005E0060AE4E1030EDB80E1D7030EDB820F
:10159000DED7030EDB84DBD7030EDB86D8D7030E42
:1015A000DB88D5D72A0EDF5C1BE106EC0FF054EC8C
:1015B0000FF010E0030EDB801E681F68130EDBCFF8
:1015C00023F0140EDBCF24F051EC13F0040E1CC0FA
:1015D000DBFF03D0130E3DEC0FF00AEC0FF00BD045
:1015E000090EDB6AABEC0FF003E01FEC10F0FAD74A
:1015F000090E3DEC0FF0030EDBB0DB982E0EDF5C26
:101600001BE10AEC0FF02A0EDF5C0BE106EC0FF099
:1016100054EC0FF003E1130E8FEC0FF00AEC0FF017
:101620000BD0090EDB6AABEC0FF003E01FEC10F0FF
:10163000FAD7090E8FEC0FF0680EDF5C07E10AECB9
:101640000FF0680EDF5C1DE1030E18D0740EDF5C36
:1016500017E07A0EDF5C14E0480EDF5C06E0540E03
:10166000DF5C03E05A0EDF5C02E1020E07D06C0E75
:10167000DF5C03E06A0EDF5C04E1010EE2EC0FF0D8
:10168000C9DBDF506E0A01E17FD31E0A01E192D16E
:10169000200A01E18FD13F0A01E149D11A0A01E193
:1016A00046D10D0A01E143D1200A01E140D13A0AB5
:1016B00001E13DD1200A01E13AD1260A01E135D10B
:1016C0000D0A01E132D11A0A01E1D9D0200A4AE01B
:1016D000300A1FE0460A0EE0250A01E083D3D95004
:1016E000F90FE96EFF0EDA20EA6E010EEE5E000ED3
:1016F000EE5AEE5AF0EC0FF0250EE66E95DB03E1A4
:10170000011C01E169D3ECEC0FF001E26BD3DB2AA1
:1017100069D3080EDB6A040EDB50010806E2040EF2
:10172000DB04B4EC0FF0DB508BDB080EDB5009E080
:10173000030EDB50010B05E172DB01E04DD3080E17
:10174000DB6A64DBEFCFDFFF64EC10F003E1011C28
:1017500001E142D3ECEC0FF001E3DB2A60DB01E1B5
:1017600041D33AD3070EDB5002080FE130EC10F002
:10177000030EF7EC0FF00E0EEECFDBFF0F0EEECFE9
:10178000DBFF100EEECFDBFF20D0F70EDBCF03F038
:10179000F80EDBCF04F0020E035E000E045AF70EC3
:1017A00003C0DBFFF80E04C0DBFF03C0E9FF04C089
:1017B000EAFFE7EC0FF0026A0E0E00C0DBFF0F0E2F
:1017C00001C0DBFF100E02C0DBFF0E0EDBCFE6FF19
:1017D0000F0EDBCFE6FF100EDBCFE6FF99EC15F026
:1017E000E552E552E552130E1DC0DBFF140E1EC07C
:1017F000DBFF060EDB5005E0130E2BEC10F001E2D0
:101800006ADB4FEC10F002E2130E37DB12EC10F043
:1018100006E0040E2BEC10F002E2050E2EDB030EA8
:10182000DBB005D0FCDA01E0D7D2080EDB6A090E86
:10183000DB6A0E0EDBCFF6FF0F0EDBCFF7FF100ECD
:10184000DBCFF8FF0800F550DF6EDF5014E055ECF9
:1018500010F011E264EC10F003E1011C01E1BCD2D4
:10186000BBDB01E3DB2A090EDB2AD9500E0FE96E40
:10187000000ECBDBE7D7D3DA01E1B4D2ADD2C6DAC2
:10188000110EEECFDBFF120EEDCFDBFF110EDBCF23
:10189000E6FF120EDBCFE6FF8BEC15F0E552E552CA
:1018A000130EF3CFDBFF140EF4CFDBFF060EDB507D
:1018B00004E0130ED0DB01E20EDB4FEC10F002E28D
:1018C000130EDBDAAFDB05E0040EC5DB02E2050E2A
:1018D000D4DA030EDBB005D0A2DA01E07DD2080E27
:1018E000DB6A090EDB6A110EDBCFE9FF120EDBCFDC
:1018F000EAFFEFCFDFFFDF5014E0D7DB12E2E4DBDB
:1019000003E1011C01E168D267DB01E3DB2A090E78
:10191000DB2A110EDB2ADBCFE9FF120EE8E3DB2A1C
:10192000E6D77DDA01E15ED257D2030EDB8E070ED9
:10193000DB0410E195DB040E5ADB0A0EEECFDBFF71
:101940000B0EEECFDBFF0C0EEECFDBFF0D0EEECF5E
:10195000DBFF6CD0070EDB5003082CE1030EDBAE7F
:101960000DD0B2DA020E76DAEFCF00F0016A026A29
:10197000036A00AE39D00168026835D0F70EDBCFBC
:1019800001F0F80EDBCF02F0020E015E000E025AEB
:10199000F70E01C0DBFFF80E02C0DBFF01C0E9FF5C
:1019A00002C0EAFFEFCF00F00A0E00C0DBFF0B0E13
:1019B000DB6A38D0070EDB50020809E1030EDBAE0C
:1019C00004D059DB02AE10D00ED055DB0DD0030E83
:1019D000DBAE12D079DA020E3DDAF9DA026A036A76
:1019E00001AE02D002680368E2DA0C0E02C0DBFF2F
:1019F0000D0E03C0DBFF1AD0F70EDBCF02F0F80E9E
:101A0000DBCF03F0020E025E000E035AF70E02C097
:101A1000DBFFF80E03C0DBFF02C0E9FF03C0EAFFF3
:101A2000D6DAC5DA0C0EDB6A0D0EDB6A060EDB5069
:101A300005E1010EF36E050EF3CFDBFF150EDB6A39
:101A4000160EDB6AD950370F006E000EDA20016ED9
:101A5000390E00C0DBFF3A0E01C0DBFF380EDB6A37
:101A6000080EDB6A0A0EAEDADF50780A12E0200AAE
:101A700010E0280A0CE0200A0AE03F0A06E00D0AFE
:101A800002E0200A08E1020E05D0080E03D0080E7D
:101A9000DF26100E97DA030EDBBE02D0DB92DB945A
:101AA000DB50800B24E08ADAD890030EEB50000A5A
:101AB00008E6000EEE5C000EEE58000EEE58000E2A
:101AC000EE5815E213DA216822682368246877EC5F
:101AD00016F00A0E18C0DBFF0B0E19C0DBFF0C0E50
:101AE0001AC0DBFF0D0E1BC0DBFF2D0E08D0030E4E
:101AF000DBA202D02B0E03D0DBA408D0200EF36EA5
:101B0000170EF3CFDBFF150EDB2A02D0170EDB6AB0
:101B1000050EDB5003E1B7D901E189D0040E006E58
:101B20002F0E016E000E026E070EDBCF03F0046A6B
:101B3000056A066A03C021F004C022F005C023F044
:101B400006C024F0D3D9AFEC16F000501824F36E81
:101B500001501920F46E02501A20F86EF4CFF7FFEE
:101B6000F3CFF6FF0800090EF5CFDBFF580EDF5C60
:101B70000FE1610EF36E090E7BD90AE3200E006EB1
:101B8000090EDBCFE7FF0050E75E090EE7CFDBFF72
:101B9000070EDBCF00F0016A026A036A0FDA00C0A9
:101BA00021F001C022F002C023F003C024F0EECFE8
:101BB0001CF0EECF1DF0EECF1EF0EFCF1FF0AFEC1C
:101BC00016F01FC0EDFF1EC0EDFF1DC0EDFF1CC0D5
:101BD000EFFF390EDBCFE9FFDB063A0EDBCFEAFF82
:101BE00001E2DB06090EDBCFEFFF150EDB2A4BD936
:101BF00095E1030EDBA61DD06F0EDF5C06E1C1D9B7
:101C000018E3150EDB285BDA14D0780EDF5C09E0F0
:101C1000580EDF5C06E0620EDF5C03E0420EDF5C24
:101C200008E1020EF36E160EF3CFDBFF02D0150EA5
:101C3000DB6A030EDB50100B0EE0040EDBCF00F06E
:101C4000050EDB50D880005406E2060EDB5003E19F
:101C5000040EDB5034DA95D90AE2050EDBCFE7FF3C
:101C6000150EDB50E75E050EE7CFDBFF02D0050E59
:101C7000DB6A040EDBCF00F0160E45D9D880005485
:101C800014E2160EDBCFE6FF150EDBCFE6FF040EE7
:101C9000DBCFE6FF050EDB50E552E75CE552D8806E
:101CA000E754E552D880E7545FD9030EDB50010BAF
:101CB0000BE1080EDB5008E0B2D801E08DD0080E31
:101CC000DB50BED8080EDB6A170EDB5007E088D960
:101CD000170EF1D903E1011C01E17ED0160EDB5095
:101CE00016E07ED9300EE66E9FD802E1011C74E04A
:101CF00077D9DFCFE6FFBEEC15F0E552E552E552AD
:101D0000F4CF01F00001F31C02E1011C65E0050EB7
:101D1000DBCF00F0160EDB50D880005409E2050E30
:101D2000DBCFE7FF160EDB50E75E050EE7CFDBFFEC
:101D3000300EE66E050ECBD94FE1390EDB2ADBCF34
:101D4000E9FF3A0E01E3DB2ADBCFEAFF090EEFCF12
:101D5000DBFFDB500EE044D9090EADD902E1011CD6
:101D60003BE0390EDB2ADBCFE9FF3A0EEDE3DB2A5D
:101D7000EBD755D831E1160EDBCFE6FF080EC3D8FE
:101D8000E552E7245DD82ED0070EDB50030A1CE095
:101D9000010A14E0030A07E07BD9DBCFEEFF020E55
:101DA000DBCFEDFF1FD0F5D8056A03AE02D0046883
:101DB00005682CD8BCD805C0EEFF14D0EAD803BE05
:101DC000046824D8B4D80ED063D9DBCFEFFF0AD093
:101DD0007BD905E1011C03E1F368F46810D0FCD85D
:101DE00001E3DB2A79D991EF0AF0010EDBCF00F095
:101DF000020EDBCF01F000C0F3FF01C0F4FF3B0E89
:101E0000E15C02E2E16AE552E16ECBD029D9020E33
:101E1000F7EF0FF061D90800F550DF6E1200200EC9
:101E2000E66E080E67EF10F0BEEC15F0E552E552D5
:101E3000E552F3CF00F0F4CF01F00001F31C1200E3
:101E4000006E016AD950010F4DD90050EE260150A5
:101E5000ED221200045E000E055AF70E04C0DBFFEF
:101E6000F80E05C0DBFF04C0E9FF05C0EAFF120061
:101E7000DBCFF4FFF350F45C1200DB50E76E040E8E
:101E8000E7CFDBFF12000A0EDBCF00F00B0EDBCF3B
:101E900001F00C0EDBCF02F00D0EDBCF03F0005093
:101EA0000110021003101200130EEECFDBFF140E10
:101EB000EDCFDBFF130EDBCF00F0140EDBCF01F014
:101EC0000001800E01141200F70EDBCF04F0F80EB3
:101ED000DBCF05F01200050EDB50E66ED950130F74
:101EE00001D9E552E750EE6EED6A12000A0EDBCF23
:101EF0001CF00B0EDBCF1DF00C0EDBCF1EF00D0E19
:101F0000DBCF1FF01200DBCFE6FF150EDBCFE6FFC5
:101F1000050EDB50E552E724E552E7241200DB50C2
:101F2000CED8010EF36E060EF3CFDBFF1200EE509B
:101F3000EFCFEAFFE96E02C0EEFF03C0EEFF04C080
:101F4000EEFF1200D9CFE6FFDACFE6FFE1CFD9FFEF
:101F5000E2CFDAFF1200DFCFE6FFE66A3BEC17F0D4
:101F6000E552E552F3501200E76E080EE7CFDBFFB3
:101F70001200EECF00F0EECF01F0EFCF02F0036AD7
:101F80001200050EDBCF00F0150EDB50D880005498
:101F90001200010EDBCF02F0020EDBCF03F0046A69
:101FA0001200E552E5CFDAFFE7CFD9FF12000A0EA3
:101FB00000C0DBFF0B0E01C0DBFF1200D9500A0F7F
:101FC00072EF10F0F36E070EF3CFDBFF1200EECFCF
:101FD00000F0EFCF01F01200010EDB2A020E12001A
:101FE000FC0EDBCFE6FFFD0EDBCFE6FF1200005E4E
:101FF000000E015AF70E00C0DBFFF80E01C0DBFF38
:1020000000C0E9FF01C0EAFF1200DA20EA6EEF2A01
:10201000EECFF6FF000EEF22EECFF7FFEF22EECF6E
:10202000F8FF1200040EDBCFE6FF130EDB50E55283
:10203000E75C9ADFDB5004DF060EDB501200090E6E
:10204000DB500A0DF350DF24D00FE76E090EE7CF07
:10205000DBFF0AEF0FF0DB50F36E050E38EF0FF0E9
:10206000F70EDBCF00F0F80EDBCF01F01200DFCF70
:10207000E6FF14EF0FF028DF030EECDEB9EF0FF0F0
:1020800066EC0AF0E552E552E552E552000912000D
:10209000BDDEEE50EFCFEAFFE96E010E1200130E27
:1020A000DB50F36E040E38EF0FF0040EDB50F36ECE
:1020B000090E38EF0FF0DBCFE6FF14EF0FF0E76EFD
:1020C000050EE7CFDBFF12008BDF37EF10F0DBCF21
:1020D000E6FF86DF40EF10F0D950F90FE96EFF0EF2
:1020E00005EF10F0E96E000EDA20EA6E1200279E6E
:1020F00008D0279E1FAE05D01E6C1F1EE86A1F2247
:10210000278E1FC019F01EC018F02B6A2A6A8E0E87
:102110001A6E1B6AE7EF12F0279E0CD0279E1FAEA7
:1021200009D01C6C1D1E1E1E1F1EE86A1D221E22C9
:102130001F22278E1FC019F01EC018F01DC02BF0E3
:102140001CC02AF09E0E1A6E1B6AE7EF12F0257E65
:10215000276A23EC13F03BEC13F027B6CBEF12F019
:1021600027A20AD027AA03D027BECBEF12F027A4BC
:10217000D7EF12F0D4EF12F027AA05D027ACD7EF93
:1021800012F0D4EF12F027A00AD027A808D027BE5B
:1021900004D027A402D0E0EF12F0E4EF12F02A6A94
:1021A0001B6A2550205C296E10E31DC02BF01EC059
:1021B00018F01FC019F020C028F022C01DF023C065
:1021C0001EF024C01FF0273A09D022C02BF023C0F4
:1021D00018F024C019F025C028F0296C279E27BCD0
:1021E000278E28C01AF027B013EF13F01A0E2960BB
:1021F00013EF13F01A6A206A27A408D01D6C1E1E64
:102200001F1E201EE86A1E221F22202227AC08D093
:102210002B6C181E191E1A1EE86A182219221A227F
:102220001C6A295207E020341F321E321D321C3234
:10223000292EF9D71D502B261E5018221F50192267
:1022400020501A221CC02AF0279E1AAE0BD02A6CEE
:102250002B1E181E191E1A1EE86A2B22182219227C
:102260001A22278E1AA006D0D880193218322B32A3
:102270002A32282A28C01AF0E7EF12F0276A23EC46
:1022800013F03BEC13F027B6CBEF12F027A205D0EA
:1022900027BACBEF12F0D2EF12F027BADEEF12F02E
:1022A00027A005D027B8CBEF12F0DEEF12F027B849
:1022B000D2EF12F01B6A7F0E20241A6EE86A1B22EE
:1022C00025501A5EE86A1B5A1A0E286E206A2A6A7E
:1022D0002B6A186A196A22501D5E23501E5A245018
:1022E0001F5A000E205A09E722501D2623501E2295
:1022F00024501F22000E202201D02A8AD8901D3699
:102300001E361F362036D8902A362B361836193608
:10231000282EE1D71F501E101D10D8A42A8AE7EFDF
:1023200012F0276A23EC13F03BEC13F027B6CBEF47
:1023300012F027A205D027B8CBEF12F0D2EF12F09F
:1023400027AA05D027B0CBEF12F0D2EF12F027B0BA
:1023500002D027A802D0DEEF12F01B6A25502024FD
:102360001A6EE86A1B227E0E1A5EE86A1B5A2A6AF7
:102370002B6A186A196A24501F02F4CF19F0F3CFA0
:1023800018F023501F02F3502B26F4501822000E91
:10239000192224501E02F3502B26F4501822000E4E
:1023A000192222501F02F3502A26F4502B22000E2D
:1023B0001822192223501E02F3502A26F4502B22F1
:1023C000000E1822192224501D02F3502A26F45020
:1023D0002B22000E1822192222501E02F4502A2607
:1023E000000E2B221822192223501D02F4502A26F7
:1023F000000E2B2218221922E7EF12F0276A23EC95
:1024000013F027B608EF12F027A20ED027B405D09C
:102410007F0E1F6EFF0E1E6E1FD0800E1F6E1E6A77
:102420001BD01F6A1E6A18D027B0FBD78F0E206002
:10243000EDD77E0E2064F5D78E0E205C05E0D89097
:102440001F321E32202AF8D727A406D01E6C1F1E6A
:10245000E86A1F221FAEE5D71200276A23EC13F0AB
:1024600027B637EF12F027A20FD027B407D07F0E80
:102470001F6EFF0E1E6E1D6E1C6E25D0800E1F6E11
:1024800001D01F6A000EF6D727B0FBD71C6A9F0E3B
:102490002060EBD77E0E2064F4D79E0E205C07E010
:1024A000D8901F321E321D321C32202AF6D727A4A4
:1024B0000AD01C6C1D1E1E1E1F1EE86A1D221E2235
:1024C0001F221FAEDED7120076EC12F027B6000CEA
:1024D00027B0000C27B4000C010C76EC12F027B6E4
:1024E000000C27B0000C27A4000C010C276A23EC79
:1024F00013F03BEC13F027B6120027AE08D027A04C
:1025000004D027A802D0278012002790120025505F
:10251000205C0BE124501F5C08E123501E5C05E1A8
:1025200022501D5C02E127801200D8A002D0278E25
:1025300010D0205025C020F0256E1F5024C01FF061
:10254000246E1E5023C01EF0236E1D5022C01DF0AD
:10255000226E2550205C10E0FF0F09E0279027B481
:1025600003D027AE2784120027AE27941200252A15
:10257000D89024322332223222501D5E23501E5A1C
:1025800024501F5A1FBEEAD7D8901D361E361F365C
:10259000202EF8D7C8D77F0E206EFF0E1F6E1E6E3E
:1025A0001D6E12007F0E27BEFF0E206E02D07F0E22
:1025B000206E800E1F6E1E6A1D6AF3D727AE04D0F0
:1025C000800E206E1F6AF7D7206A1F6AF4D7195051
:1025D00018102B102A10F8E01BBEF0D719BE0CD033
:1025E0001A501B10EBE0D8902A362B3618361936C5
:1025F0001A06D8A01B06F2D71B50D4E11A28D2E045
:102600002AAE11D07F0E2A1402E12BA00CD02B2A67
:10261000E86A1822192207E3D880193218322B32BF
:102620001A2A1A28BFE01A50C9E02BC01DF018C0A2
:102630001EF019341F6E1A30206E1F32209E27BEE6
:10264000208ED1EF12F01F36203602E32784277E3A
:1026500006E12780206A1F6A1E6A1D6A1200202870
:1026600003E0D8801F321200D8901F3202E1278287
:102670001200278612002436253602E3278C277E97
:1026800006E12788256A246A236A226A120025281F
:1026900003E0D88024321200D8902432EAE1278A5D
:1026A00012001FC02BF01EC02AF01E502302F4CFD0
:1026B0001DF0F3CF1CF01F502402F4CF1FF0F3CF16
:1026C0001EF02302F3501D26F4501E22E86A1F223A
:1026D0002A502402F3501D26F4501E22E86A1F22BD
:1026E00024AE77EF13F02A501E5E2B501F5A2BAEEC
:1026F000000C23501E5E24501F5A000CD9CFE6FF59
:10270000DACFE6FFFA0EE3CFD9FFFB0EE3CFDAFF15
:10271000FD0EE35209E72D0EDE6EFC0EE31EE32AEA
:10272000FD0ED8B4E306E31EE652E652E652FD0E75
:10273000E124E76EFF0EE220E46EE652F70EE3CFEF
:10274000E6FFF70EE3CFE6FFEEEC13F0F90EE1241F
:10275000E96EFF0EE220EA6EDEEC13F00AE1DBEC3C
:1027600013F009E1DEEC13F008E1DBEC13F007E114
:1027700008D0E9EC13F0E4EC13F0E9EC13F0E4EC2E
:1027800013F0E9EC13F0DE6AF90EE126FF0EE22207
:10279000FF0EE3CFDAFFE552FF0EE3CFD9FFE5529C
:1027A000FC0EE124E96EFF0EE220EA6EEECFF3FFAD
:1027B000EFCFF4FF1200EF380F0B1200EF500F0BAA
:1027C00002E1EE52D8841200EF380F0B300FDE6EAC
:1027D0001200EE500F0B300FDE6E1200FC0EE3CF36
:1027E000E9FFFD0EE3CFEAFF100EE66EEE6AEE6A39
:1027F000EF6AD890FD0EE336FE0EE336ED36ED3689
:10280000EF36FF0EE30609E00FEC14F0EE520FEC8A
:1028100014F0EE520FEC14F0EDD7E56E1200030E3B
:10282000EF24E8B6EF6E300EEF24E8BEEF6E000C3A
:10283000D9CFE6FFDACFE6FFF80EE3CFD9FFF90EE6
:10284000E3CFDAFFE652E652E652E652E652FB0EDC
:10285000E124E76EFF0EE220E46EE652F30EE3CFD2
:10286000E6FFF30EE3CFE6FFF30EE3CFE6FFF30E52
:10287000E3CFE6FF9DEC14F0F50EE124E96EFF0EC8
:10288000E220EA6E8AEC14F019E18DEC14F018E104
:102890008AEC14F017E18DEC14F016E18AEC14F0D8
:1028A00015E18DEC14F014E18AEC14F013E18DECD9
:1028B00014F012E18AEC14F011E112D093EC14F050
:1028C00098EC14F093EC14F098EC14F093EC14F0F2
:1028D00098EC14F093EC14F098EC14F093EC14F0E2
:1028E00098EC14F0DE6AF50EE126FF0EE222FF0EF0
:1028F000E3CFDAFFE552FF0EE3CFD9FFE552FA0E40
:10290000E124E96EFF0EE220EA6EEECFF3FFEFCF97
:10291000F4FF1200EF380F0B1200EF500F0B02E123
:10292000EE52D8841200EF380F0B300FDE6E12001B
:10293000EE500F0B300FDE6E1200FA0EE3CFE9FF00
:10294000FB0EE3CFEAFF200EE66EEE6AEE6AEE6A59
:10295000EE6AEF6AD890FB0EE336FC0EE336FD0E0E
:10296000E336FE0EE336ED36ED36ED36ED36EF3678
:10297000FF0EE3060FE0CCEC14F0EE52CCEC14F0BA
:10298000EE52CCEC14F0EE52CCEC14F0EE52CCEC57
:1029900014F0E1D7E56E1200030EEF24E8B6EF6EF7
:1029A000300EEF24E8BEEF6E000C0E0EF66E000E39
:1029B000F76E000EF86E0F010900F550056F090063
:1029C000F550066F03E1056701D03DD00900F550D1
:1029D000006F0900F550016F0900F550026F090002
:1029E0000900F550E96E0900F550EA6E090009008A
:1029F0000900F550036F0900F550046F0900090044
:102A0000F6CF07FFF7CF08FFF8CF09FF00CFF6FF9B
:102A100001CFF7FF02CFF8FF0F01035302E1045388
:102A200007E00900F550EE6E0307F8E20407F9D756
:102A300007CFF6FF08CFF7FF09CFF8FF0F01050713
:102A4000000E065BBFD71200D9CFE6FFDACFE6FF54
:102A5000E1CFD9FFE2CFDAFFE652E652E652E65284
:102A6000D950F90F006EFF0EDA20016E00C0DEFFB4
:102A7000DD6EDECFE6FFDDCFE6FFF90EDBCFE6FF52
:102A8000FA0EDBCFE6FFFB0EDBCFE6FFFC0EDBCF63
:102A9000E6FFFD0EDBCFE6FF7CEC0AF0006E070ED2
:102AA000E15C02E2E16AE552E16E0050020EF3CF12
:102AB000DBFF030EF4CFDBFF020EDBCF00F0030ED3
:102AC000DBCF01F000C0F3FF01C0F4FF040EE15CB6
:102AD00002E2E16AE552E16EE552E5CFDAFFE7CFC7
:102AE000D9FF1200FB0EE3CFF6FFFC0EE3CFF7FF9A
:102AF000FD0EE3CFF8FFFE0EE3CFE9FFFF0EE3CFBD
:102B0000EAFFE9CFF3FFEACFF4FF0900F5CFEFFFCB
:102B1000EE66FBD71200FE0EE3CFE9FFFF0EE3CF18
:102B2000EAFFF36AF46AEE5203E0F34AF42AFBD7B1
:102B30001200FF0EE3CFF8FFE552FF0EE3CFF7FFE1
:102B4000E552FF0EE3CFF6FFE552E66AE66AE66A73
:102B50000900F55209E0FD0EE32A05E1FE0EE32A25
:102B600002E1FF0EE32AF4D7FD0EE3CF1DF0FE0EC7
:102B7000E3CF1EF0FF0EE3CF1FF01200D9CFE6FF28
:102B8000DACFE6FFE1CFD9FFE2CFDAFFFB0EDBCFF2
:102B900000F0FC0EDBCF01F00001800E01141AE101
:102BA000FB0EDBCFE9FFFC0EDBCFEAFFEECFF3FF3E
:102BB000EDCFF4FFEE2A000EEF22F3CFE9FFF4CFC2
:102BC000EAFFFD0EDBCFEFFFEF50016AF36E01C0AD
:102BD000F4FF10D0FB0EDB50FE0806E1FD0EDBCF4C
:102BE000E6FF6BEC17F005D0FD0EDBCFE6FF03EC44
:102BF00000F0E552E552E5CFDAFFE7CFD9FF12004A
:102C00002E2E2E004F7363696C6C20696E74657292
:102C10006E652031364D687A200D0A004331383A0E
:102C20002031384632364B32325F4343505F647551
:102C30007265652E630D0A0045534320706F7572EF
:102C400020736F727469720D0A004361707475723B
:102C5000652043435031207375722070696E205295
:102C600043320D0A00557365203420726973696E12
:102C70006773204564676573200D0A00D9CFE6FFAE
:102C8000DACFE6FFE1CFD9FFE2CFDAFFAC6AAB6A79
:102C9000FD0EDBB0AC88DBA202D0AC8CAB8CDBB41D
:102CA000AC8EDBA602D0AB8801D0AB8ADBB8AC849B
:102CB000DBBAAB86DBAC02D09D8A01D09D9ADBAE3D
:102CC00002D09D8801D09D98FB0EDB50AF6EFC0EAC
:102CD000DBCF01F001C000F0016A0050B06EAC8A99
:102CE000AB8EE552E5CFDAFFE7CFD9FF12001C50DB
:102CF0002102F3CF18F0F4CF19F02202F350192675
:102D0000000EF4201A6E1C502302F3501A26000EF7
:102D1000F4201B6E1C502402F3501B261D50210270
:102D2000F3501926F4501A22000E1B221D502202C5
:102D3000F3501A26F4501B221D502302F3501B2679
:102D40001E502102F3501A26F4501B221E5022025C
:102D5000F3501B261F502102F3501B2612001B6A42
:102D60001A6A196A186A200EE76ED8901C361D364A
:102D70001E361F36183619361A361B362150185C87
:102D80002250195823501A5824501B5809E3215037
:102D9000185E2250195A23501A5A24501B5A1C2AC2
:102DA000E72EE4D71200D9CFE6FFDACFE6FFE1CF76
:102DB000D9FFE2CFDAFFE652F20E0001FE17ABAC0C
:102DC00003D0FE91ABB0FE81ABB4FE85ABB2FE8703
:102DD000AE50DF6EDF50E552E552E5CFDAFFE7CFC8
:102DE000D9FF1200D9CFE6FFDACFE6FFE1CFD9FF56
:102DF000E2CFDAFFE652E652FC0EDBCFDEFFDBCF9E
:102E0000DDFF010EDB50CF6EDF50CE6EE552E55296
:102E1000E552E5CFDAFFE7CFD9FF1200D9CFE6FFC1
:102E2000DACFE6FFE1CFD9FFE2CFDAFFACAC04D0D6
:102E3000AC900001FEB3AC80FD0EDB50AD6EE552F0
:102E4000E5CFDAFFE7CFD9FF12001B6A1A6A100E2E
:102E5000E76ED8901E361F361A361B3623501A5C82
:102E600024501B5805E323501A5E24501B5A1E2A77
:102E7000E72EF0D71200F36AF46AFF0EE124E96E40
:102E8000FF0EE220EA6EED6607D02F0EEF6404D04D
:102E90003A0EEF6001D0F32A1200380EF36E00EE06
:102EA00000F00F0E01D81200EA6002D0EE6AFCD7E3
:102EB000F350E9601200EE6AFCD71EEE00F02EEE31
:102EC00000F0F86A279CD5EC14F08BEC17F02FEC8F
:102ED00008F0FBD71200FF0EE350ACBA04D0AF6A83
:102EE000AB8EAC8A949CACA2FED7AD6EF36EF46A46
:102EF0001200463D202573203B2052706D3D202559
:102F0000730D0A0030313233343536373839616267
:102F10006364656600FF1200002C042C1C2C382C06
:102F20004A2C652C31384632364B32322065737369
:102F30006169206D657375726520647572656520C1
:102F40007669612043435031202870696E205243D6
:102F50003229200D0A0000000000000000000000DF
:102F600000000000313233343536373839303132F1
:102F7000333435360030303030303030303030306F
:102F800030303030303030303030303000050505F2
:102F900005050505050505050505050505050505E1
:102FA00005050505050505050505050505050505D1
:102FB000050505050500FFFFFFFFFFFFFFFFFFFF02
:102FC000FFFFFFFFFFFFFFFFFFFFFFFFFFFFFFFF11
:102FD000FFFFFFFFFFFFFFFFFFFFFFFFFFFFFFFF01
:102FE000FFFFFFFFFFFFFFFFFFFFFFFFFFFFFFFFF1
:102FF000FFFFFFFFFFFFFFFFFFFFFFFFFFFFFFFFE1
:0200000400F00A
:1000000050726F6A65743A2031384632364B32325C
:100010005F4343505F64757265652E6320200D0059
:10002000496E697420506F725420436F6D20525393
:100030003233322031393230306264732E200D0079
:100040002E2E2E2E2E2E2E2E2E2E2E2E2E2E2E2ED0
:1000500020203C4553433E206578697420200D00E4
:1000600041766563205541525420484152445741DE
:1000700052452E2E2E2E2E2E2E2E2E2E2E200D00C2
:100080002020202020202020202020202020202070
:1000900020202020202020202020202020200D0093
:1000A0007061756C666A756A6F40667265652E660A
:1000B00072202032332F30392F32303133200D006F
:1000C0004D504C4142204944452056382E3930206D
:1000D000204331382076332E34352E30310D000058
:1000E0002020202020202020202020202020202010
:1000F000202020202020202020200D0A00000000A9
:10010000FFFFFFFFFFFFFFFFFFFFFFFFFFFFFFFFFF
:10011000FFFFFFFFFFFFFFFFFFFFFFFFFFFFFFFFEF
:10012000FFFFFFFFFFFFFFFFFFFFFFFFFFFFFFFFDF
:10013000FFFFFFFFFFFFFFFFFFFFFFFFFFFFFFFFCF
:020000040030CA
:0E0000000028193C009D84000FC00FE00F4047
:020000040020DA
:08000000FFFFFFFFFFFFFFFF00
:00000001FF
